:100000000C9400030C9438030C9438030C943803BC
:100010000C9438030C9438030C9438030C94380374
:100020000C9438030C9438030C94BB250C948D2647
:100030000C94AF200C9438030C9438030C943803C0
:100040000C9438030C9438030C9438030C94380344
:100050000C9438030C9437210C9438030C94380317
:100060000C9438030C9438030C9438030C94380324
:100070000C9438030C9438030C9438030C94380314
:100080000C9438030C9438030C9438030C94380304
:100090000C9438030C9438030C9438030C943803F4
:1000A0000C9438030C9438030C94380367056705E7
:1000B00093059305FB051906310731072406BD0694
:1000C000CE06CE06FA2621271928212719286D27C2
:1000D00090271928E727F62729001E001F00200077
:1000E00021002200230024002500260027002D00E7
:1000F0002E0000002A004A002B00000014001A0005
:100100000800150017001C0018000C001200130056
:100110002F00300031004B003900000004001600B1
:10012000070009000A000B000D000E000F0033004D
:100130003400280000004E00E10000001D001B00FC
:1001400006001900050011001000360037003800C5
:100150000000E50052004D00E000E300E200000076
:10016000000000002C00000000000000E600E70096
:100170000151500051004F0035003A003B003C0057
:100180003D003E003F00400041004200430044006B
:10019000450000004C004900010000000100520031
:1001A0000100010001000100010046004700480075
:1001B0000100010001000100010000005000510099
:1001C0004F000100010001000100010001000100D9
:1001D0000100010000000100010000000100010019
:1001E0000100010001000100010001000100010007
:1001F000000001004B000100005C01000100000054
:1002000000000000010000000000000001000100EB
:1002100001004A004E004D000100010001000100F4
:1002200001000100010001000100010001000100C6
:1002300001000000010001000100000001000100B8
:1002400001000100010001000100010001000100A6
:100250000100010001000100010000000100010097
:100260000100010001000100010001000100010086
:100270000100010000000100010000000100010078
:100280000100010001000100010001000100010066
:10029000000001004B00010001000100010000000E
:1002A000000000000100000000000000010001004B
:1002B000010001000100010000047F3F1F643214AF
:1002C000643214783C1E1E140A0522232526282990
:1002D0002A2C2D2F3032333536383A3B3D3E4042C2
:1002E000434547494A4C4E5051535557595A5C5E05
:1002F0006062646668696B6D6F71737577797B7D19
:100300007F81838587898A8C8E90929496989A9C17
:100310009E9FA1A3A5A7A8AAACAEAFB1B3B4B6B82F
:10032000B9BBBCBEBFC1C2C3C5C6C7C9CACBCCCD91
:10033000CED0D1D2D2D3D4D5D6D7D7D8D9D9DADA6C
:10034000DBDBDBDCDCDCDCDCDDDDDDDDDCDCDCDCEC
:10035000DCDBDBDBDADAD9D9D8D7D7D6D5D4D3D220
:10036000D2D1D0CECDCCCBCAC9C7C6C5C3C2C1BFFE
:10037000BEBCBBB9B8B6B4B3B1AFAEACAAA8A7A562
:10038000A3A19F9E9C9A98969492908E8C8A89871E
:100390008583817F7D7B79777573716F6D6B6968FC
:1003A000666462605E5C5A5957555351504E4C4AD0
:1003B0004947454342403E3D3B3A3836353332307B
:1003C0002F2D2C2A292826252322FFAA7F554000DD
:1003D0000101010101010101010202020202020206
:1003E00002020303030303030303040404040404D9
:1003F000040505050505060606060607070707079F
:1004000008080808090909090A0A0A0B0B0B0C0C51
:100410000C0D0D0D0E0E0E0F0F0F101011111112ED
:100420001213131414151516161717181819191A6C
:100430001A1B1B1C1D1D1E1E1F20202122222324CF
:1004400024252626272829292A2B2C2D2D2E2F300E
:10045000313232333435363738393A3B3C3D3E3F22
:10046000404142434445464748494A4C4D4E4F500F
:10047000515354555658595A5B5D5E5F61626465CD
:100480006668696B6C6D6F7072737577787A7B7D57
:100490007E8082838587888A8C8E8F9193959698AB
:1004A0009A9C9EA0A2A3A5A7A9ABADAFB1B3B5B7C7
:1004B000BABCBEC0C2C4C6C9CBCDCFD1D4D6D8DB9E
:1004C000DDDFE2E4E7E9EBEEF0F3F5F8FAFDFF0E2D
:1004D00003570061006C0074006500720000001298
:1004E00003530077006900660074007200610078B1
:1004F0000000000403090409023B00020100A0FA05
:100500000904000001030101000921110100012279
:1005100040000705810308000109040100010300F0
:100520000000092111010001227B00070582032040
:1005300000011201000200000008D80464E9010073
:100540000102000105010902A10185020901A100C2
:100550000509190129081500250195087501810271
:100560000501093009311581257F9502750881063D
:1005700009381581257F950175088106050C0A3813
:10058000021581257F950175088106C0C005010906
:1005900080A101850319012AB700150126B700952E
:1005A0000175108100C0050C0901A1018504190124
:1005B0002AA002150126A002950175108100C00530
:1005C000010906A101050719E029E7150025019594
:1005D0000875018102950175088101050719002937
:1005E000FF150026FF009506750881000508190112
:1005F0002905950575019102950175039101C000CA
:1006000011241FBECFEFDAE0DEBFCDBF04B603FE7C
:1006100018C08091250390912603A0912703B091E3
:1006200028038730904BA740B04B59F41092250314
:10063000109226031092270310922803E0E0F8E3BB
:10064000099511E0A0E0B1E0E8E9F2E502C005900B
:100650000D92A83DB107D9F723E0A8EDB1E001C0A4
:100660001D92A532B207E1F70E9459130C944A2952
:100670000C94000081E0089581E008950C943C03FF
:1006800008950C9440031F93CF93DF9300D000D0C4
:100690001F92CDB7DEB749835A836B833091DB015C
:1006A00089819A81311114C0662359F0222349F0BF
:1006B0000E946E09182F682F89819A810E9417095C
:1006C00003C00E944209182F69817A81812F04C0DA
:1006D0000E946E0969817A810F900F900F900F90A0
:1006E0000F90DF91CF911F910C94C210FC01262F27
:1006F000408151816281738184810C94430381E044
:100700000895CF93DF93EC0160E00E947603BE0171
:10071000DF91CF910C9441030C940A120C940612B1
:1007200008950E94C1070E9490032FEF84E39CE08C
:10073000215080409040E1F700C000000C945D2102
:100740000F931F93CF93DF938C0161E00E94760398
:10075000EC01B8010E943E03882309F444C0B801AB
:10076000CE010E947A1F8823F1F1B801CE010E94C8
:100770001B1D8823C1F1B801CE010E94D61E88231B
:1007800091F1B801CE010E94211C882361F1F8018A
:100790008281882309F1CB358DE5D807C1F050F46B
:1007A000C115FCE5DF0781F0CF3DDC45A9F40E94CF
:1007B000A50E19C0CC35EDE5DE0761F0CD35DD4580
:1007C00059F40E94E80D08C00E9491030CC00E94D9
:1007D000F10D02C00E94F40DC801DF91CF911F916D
:1007E0000F910C943A0380E0DF91CF911F910F910C
:1007F00008950E9491200C9412040E9415040C94F8
:10080000972008950C94010481E008950C94040449
:100810000895CF93C82F0E9402048C2F0E940604D3
:10082000CF91089580E00C9409040E94D61F0C9487
:1008300009040E94D61F9091DA01891721F0809354
:10084000DA010C9409040895CF93DF93CDB7DEB796
:100850002B970FB6F894DEBF0FBECDBF4F835887DE
:1008600069877A878B8761110E94340D9E012F5F03
:100870003F4F86E0F90111928A95E9F785E0FE0184
:100880003796D90101900D928A95E1F789819A8175
:100890004C815D81452B31F09F3F31F491E08F3FDA
:1008A00019F403C091E001C090E090FF09C04981B4
:1008B0005A816B817C818D819E810E94550C05C07F
:1008C000C9010E947F038111F2CF2B960FB6F894D5
:1008D000DEBF0FBECDBFDF91CF910895FC018081B7
:1008E00091810E94B0090895CF93882309F450C0E4
:1008F000C82F8CEF8C0F813AD0F46C2F80910201BD
:10090000909103010E943320882349F06C2F80913D
:100910000201909103010E946B200E94560D6C2FE2
:1009200080910201909103010E9469200CC080E235
:100930008C0F883058F4C77081E001C0880FCA95C9
:10094000EAF70E94170DCF910C94560DEBE5EC0FD2
:10095000E33040F4F0E0E65AFE4F808190E0CF9122
:100960000C94FB1FE8E5EC0FE73150F4F0E0EE0FDC
:10097000FF1FE45DFE4F80819181CF910C94112087
:10098000CD3E30F08C2F0E94DE13CF910C94B0142A
:10099000CF910895882389F19CEF980F913A40F404
:1009A000682F80910201909103010E946B200DC07D
:1009B00090E2980F983058F4877091E001C0990F39
:1009C0008A95EAF7892F0E941D0D0C94560D9BE520
:1009D000980F933020F480E090E00C94FB1F98E592
:1009E000980F973120F480E090E00C9411208D3E18
:1009F00020F00E9439140C94B01408951F93CF93E3
:100A0000DF93182FEB010E947404209741F08FE9C7
:100A10009FE00197F1F700C000002197F6CF812FEA
:100A2000DF91CF911F910C94CA04893319F060E0D3
:100A300070E002C060E570E00C94FE04882321F0B1
:100A40000E94170D0C94560D0895882321F00E94E2
:100A50001D0D0C94560D0895CF92DF92EF92FF92E8
:100A60000F931F93CF93DF937C01D62FC72FFC01E9
:100A70001281058102950F700E940D0D8823B9F037
:100A80001123A9F08C2F807F803421F080E28D0F1C
:100A9000883068F08091B20282FD09C082E00E9435
:100AA000B60D0E940D0D91E0D82ED92601C0D12C93
:100AB000CC2EC2948FE0C8228C2D90E08C30910512
:100AC00008F0CFC1FC01EA5AFF4F0C94A5288C2FE7
:100AD000807FCF70882311F0C295C07F112399F0D9
:100AE000CC2309F4AAC180E28D0F883010F0D11117
:100AF00004C08C2F0E94170D03C08C2F0E94270D5D
:100B00000E94560D9AC18D2F0E94CA04CC2309F46D
:100B1000A8C180E28D0F883038F1DD2329F18C2FB8
:100B20000E942D0D24C08C2F807FCF70803211F059
:100B3000C295C07FDD2319F0D130A1F13DC0809175
:100B4000B20282FF17C0112349F0CC2329F08C2F69
:100B50000E94170D0E94560D80E070C180E00E9437
:100B6000CA04CC2309F47DC18C2F0E941D0D0E9464
:100B7000560D77C1112371F0002341F0013031F49B
:100B80000E94370D8C2B0E943F0D6BC10E94370DC8
:100B90008C2B1DC0002319F0013009F462C10E94A2
:100BA0004C0D25C0112321F0063008F05AC10EC0AB
:100BB000053008F056C11BC0112361F0002331F04D
:100BC000F701858180FF39C18F7085838C2F0E944A
:100BD0001E0547C1002359F0D93309F03FC1FFEF8B
:100BE00007EE13E0F15000401040E1F735C18C2FC3
:100BF0000E94250536C18C2F86958695837019F045
:100C0000813061F02EC1112321F08D2F9C2F937024
:100C100002C080E090E00E94FB1F2BC1112321F055
:100C20008D2F9C2F937002C080E090E00E941120D5
:100C300020C18D2F112319F00E94DE1302C00E94E3
:100C400039140E94B01415C18C2F837009F047C06D
:100C500011110BC12D2F229526952770220F220FDF
:100C60006D2F6F70862F90E0A0E0B0E0022E04C0E0
:100C7000880F991FAA1FBB1F0A94D2F7D4FF10C078
:100C80004FE050E060E070E004C0440F551F661F65
:100C9000771F2A95D2F7409550956095709503C0BF
:100CA00040E050E0BA01C695C695C3708A019B0129
:100CB000082B192B2A2B3B2BC901B801C23049F054
:100CC00058F4C13019F00E942D08CFC00E941B08B3
:100CD000CCC00E943F08C9C00E941908C6C0112399
:100CE00019F08C2F817001C08695882309F4BDC04E
:100CF0002D2F229526952770220F220F6D2F6F70B2
:100D0000862F90E0A0E0B0E0022E04C0880F991F6B
:100D1000AA1FBB1F0A94D2F7D4FF10C04FE050E0C7
:100D200060E070E004C0440F551F661F771F2A95CE
:100D3000D2F7409550956095709503C040E050E023
:100D4000BA01C695C695C3708A019B01082B192B61
:100D50002A2B3B2BC901B801C23049F058F4C130ED
:100D600019F00E94F20881C00E94E0087EC00E9433
:100D700004097BC00E94530878C0CF70112339F05A
:100D80008C2F0E9479088D2F0E941E056EC08D2F1A
:100D90000E9425058C2F0E949A0867C0D23F21F13E
:100DA00028F4D03F41F0D13FC1F043C0D33F19F107
:100DB000D43F79F03EC0112341F0053008F051C016
:100DC0008C2F8F710E94BF084CC0063008F049C0BC
:100DD000F7CF8091B20282FF18C0112339F08C2F17
:100DE0008F710E9479083DC01123C9F38C2F8F7138
:100DF0000E949A0836C0112329F08C2F8F710E940F
:100E000064082FC00E945F082CC0112349F0CF71E5
:100E10008C2F0E94790863E08C2F0E949B0D21C0CB
:100E200081E00E94B60D0230E0F082E00E94B60D33
:100E300018C0112331F0002391F28D2F0E94740409
:100E400010C0002399F2D93349F41FEF27EE33E0A5
:100E5000115020403040E1F700C000008D2F0E946B
:100E6000CA0488EF8C0D843020F40E94D61F0E94A3
:100E70000904DD20C9F00E94090D80FD15C0F701AD
:100E800012820E94030D0E947908C7010E94750713
:100E90000E94030DDF91CF911F910F91FF90EF9072
:100EA000DF90CF900C949A08DF91CF911F910F9112
:100EB000FF90EF90DF90CF9008950F931F93CF9303
:100EC000DF93EC01688179818A810E94BB098C01E2
:100ED0000E9416090E940708B801CE010E942C0545
:100EE000DF91CF911F910F910895CF93DF93EC0184
:100EF000988189812B813C81232B31F08F3F31F404
:100F000081E09F3F19F403C081E001C080E080FDD3
:100F10001DC0CE010E94A003811110C00E940D0DC2
:100F20008823A1F08A81882389F08091B20282FD12
:100F30000DC082E0DF91CF910C94B60DCE010E94DE
:100F40005D07CE01DF91CF910C948103DF91CF91AA
:100F5000089580E090E00E94FB1F80E090E00E94F6
:100F600011200E94340D0E94560D0E94E1150C9430
:100F7000B01480910201909103010E946D200C94A5
:100F8000A9070E94240D0C94B90792959F70963082
:100F900079F010F4925001C09A50923068F4803F7A
:100FA00069F018F4883E40F409C0843F29F406C073
:100FB000883E20F0813F11F080E0089581E008959F
:100FC000FC01808191810E94B0090E94C5070895AB
:100FD000CF93DF9300D000D01F92CDB7DEB70F9034
:100FE0000F900F900F900F90DF91CF910895CF93B6
:100FF000DF9300D000D000D0CDB7DEB726960FB675
:10100000F894DEBF0FBECDBFDF91CF910895089554
:1010100008950C9408080C9409080E940B0860932A
:1010200012027093130280931402909315020C9491
:10103000A9070C940D080F931F93009112021091B1
:1010400013022091140230911502602B712B822B18
:10105000932B1F910F910C940D080F931F930091E8
:101060001202109113022091140230911502602394
:101070007123822393231F910F910C940D080F93DA
:101080001F930091120210911302209114023091CB
:10109000150260277127822793271F910F910C94C7
:1010A0000D080C9408080E94510860930E0270937A
:1010B0000F0280931002909311020C94A90760E034
:1010C00070E0CB010C9453080F931F9341E050E064
:1010D00060E070E08A019B0104C0000F111F221F15
:1010E000331F8A95D2F7C901B8011F910F910C9453
:1010F00053080F931F9341E050E060E070E004C09C
:10110000440F551F661F771F8A95D2F780910E02F4
:1011100090910F02A0911002B09111028A019B01DF
:10112000082B192B2A2B3B2BC901B8011F910F91BA
:101130000C9453080F931F9341E050E060E070E07F
:1011400004C0440F551F661F771F8A95D2F740953C
:1011500050956095709580910E0290910F02A0912C
:101160001002B09111028A019B01082319232A233E
:101170003B23C901B8011F910F910C9453080F93A1
:101180001F9341E050E060E070E004C0440F551F41
:10119000661F771F8A95D2F780910E0290910F02F9
:1011A000A0911002B09111028A019B010827192712
:1011B0002A273B27C901B8011F910F910C945308AE
:1011C0000F931F9300910E0210910F0220911002B5
:1011D00030911102602B712B822B932B1F910F9159
:1011E0000C9453080F931F9300910E0210910F025D
:1011F00020911002309111026023712382239323E6
:101200001F910F910C9453080F931F9300910E029E
:1012100010910F0220911002309111026027712766
:10122000822793271F910F910C945308089520E172
:10123000929F800D1124E82FE695E695E69587703C
:1012400051E001C0550F8A95EAF785E0E89FF0016B
:101250001124E452FE4F20E030E070E04081CB01E9
:10126000022E02C0969587950A94E2F781708195C7
:1012700084278523842781932F5F3F4F25303105B5
:1012800069F7089520E1929F800D1124682F6695DB
:1012900066956695982F977085E0689FB001112438
:1012A00040E050E080E0FB01E40FF51FE452FE4F08
:1012B000208130E0092E02C0369527950A94E2F786
:1012C00021703327042E01C0220F0A94EAF7822BE3
:1012D0004F5F5F4F4530510531F70895BF92CF9270
:1012E000DF92EF92FF920F931F93CF93DF938C01C6
:1012F000C0900E02D0900F02E0901002F090110208
:101300008091120290911302A0911402B0911502E3
:10131000C82AD92AEA2AFB2ACFE1D0E0D701C601A0
:101320000C2E04C0B695A795979587950A94D2F789
:1013300080FD04C0219790F7B12C07C0BC2EB801E6
:101340008C2F0E94D7100197A9F38B2DDF91CF919D
:101350001F910F91FF90EF90DF90CF90BF90089575
:10136000CF93DF93EC010E946E09BE010E94D7105B
:10137000DF91CF9108951F93CF93DF93EB0190916D
:10138000DB01992321F0CB010E94B00913C088230F
:1013900049F0CB010E946E09182F682FCE010E94E0
:1013A000170904C0CB010E944209182FBE01812FEA
:1013B0000E94D710DF91CF911F9108951F93CF9373
:1013C000DF93C091160216E080911702C81799F0BA
:1013D000D0E01C9FF0011D9FF00D1124E85EFD4F31
:1013E0004081518162817381848195810E94F707D8
:1013F0002196C770E9CFDF91CF911F910895409159
:1014000048025091490260914A0270914B028091CA
:101410004C0290914D020C94F707EF92FF920F93BC
:101420001F93CF93DF9380914D0282958F7009F0C7
:1014300065C080914A02882309F460C08091160239
:10144000F0901702109148020091490260914B02FE
:1014500070914C0291E01F3F09F090E0C0910001B3
:10146000D0910101292F96E0E92E8F1509F446C08D
:101470006115710521F00F3F21F030E003C031E02C
:1014800001C0322F90E030FD36C0E89EF001E99EA9
:10149000F00D1124DF01A85EBD4F11963C9111970C
:1014A000301329C03C91311326C012963C911297FB
:1014B000311121C013964D915C911497461B570B27
:1014C0004C175D07C0F480914D028F70806180934E
:1014D0004D02E35EFD4F80818F708061808388E4E0
:1014E00092E00E947507DF91CF911F910F91FF90BD
:1014F000EF900C94DE0901968770B7CFDF91CF9102
:101500001F910F91FF90EF9008959F92AF92BF921D
:10151000CF92DF92EF92FF920F931F93CF93DF93BF
:10152000CDB7DEB761970FB6F894DEBF0FBECDBF63
:101530008C0185E0F801DE011D9601900D928A95DF
:10154000E1F7D8011296EC9090914802E09149029F
:1015500020914B0230914C022115310531F0EF3FC3
:1015600031F481E09F3F19F403C081E001C080E0C5
:10157000B82FB1709B2E80FD47C1D8014C911196B8
:101580005C9111971396AD90BC90149788E4C82E87
:1015900082E0D82EF0904A02B501621B730B2091B5
:1015A000000130910101FF2009F4D9C080914D0262
:1015B0006217730708F095C0282F207F09F052C0EA
:1015C0005E1313C0491311C0FE2CE1100EC08F70C2
:1015D000806180934D020E94FF09C6010E94750739
:1015E00080914D02F80185834DC1AB2831F05F3FFA
:1015F00031F481E04F3F19F403C081E001C080E085
:1016000080FD03C081E08E2502C080E090E0F82FCD
:10161000F170FF2E80FF1CC08091160220911702EE
:1016200036E0821709F40BC190E0389FF001399F32
:10163000F00D1124E85EFD4F6181561306C06081F4
:10164000461303C06281E61203C001968770E9CF9A
:10165000FE2CEE2009F416C180914D02816080932A
:101660004D0254C05E1306C0491304C0E11002C00D
:10167000F80199C0C8010E94E007882361F1EE20BB
:1016800051F120914D02822F82958F7090E0029748
:1016900074F0809148029091490298878F8319864F
:1016A000BB86AA862C87CE0107960E94750786E026
:1016B000F801A8E4B2E001900D928A95E1F70E944A
:1016C0000D0A0E94FF090AC05E1711F1C8010E94AD
:1016D000E00781112CC0C8010E947507FF24F39414
:1016E000D1C0282F207F81F77A2DB98AA88A6E2D44
:1016F00089890E94E80788E492E00E94750786E0E5
:10170000D6011D928A95E9F70E94FF09F12CBAC013
:101710004913DCCFE110DACFF8018583C8010E94BC
:10172000750786E0D6011D928A95E9F7ABC0EE20D9
:1017300091F220914D02822F82958F7090E0029756
:101740000CF4B5CF80914802909149029A83898325
:101750001B82BD82AC822E83CE010196A6CF62177A
:10176000730708F044C0FE2CEE2009F4B4CF5E13DA
:1017700030C049132EC020914D0220FD21C0822F80
:1017800082958F70482F50E041155105C9F0F8013E
:1017900025834F30510541F08F5F982F9295907FB0
:1017A000822F8F70892B8583C8010E94750786E080
:1017B000F801A8E4B2E001900D928A95E1F73CC0EF
:1017C00086E0F801A8E4B2E001900D928A95E1F775
:1017D00059C0C8010E94E007811169CF80914D0274
:1017E000816080934D02C8010E9475074BC07A2D1D
:1017F000B98AA88A6E2D89890E94E80786E0D601F9
:101800001D928A95E9F718C0EE2009F464CFC8014B
:101810000E94E007F82E882309F45DCF86E0F801E6
:10182000A8E4B2E001900D928A95E1F788E492E095
:101830000E946E040E940D0A0E94FF0923C04D877A
:101840005E878D859E850E94B009292F22952F7075
:10185000223028F49F7039F0811105C00BC024306C
:1018600028F49F7049F4805E883020F0C8010E94FF
:1018700075079F2CF92C06C0D80115969C91907F76
:1018800091F7F8CF8F2D61960FB6F894DEBF0FBE9B
:10189000CDBFDF91CF911F910F91FF90EF90DF901F
:1018A000CF90BF90AF909F9008951F93CF93DF93F9
:1018B000CDB7DEB72C970FB6F894DEBF0FBECDBF05
:1018C0004F83588769877A878B879C87CE010796D5
:1018D0000E94850A8823D1F09F8188852A853B85CF
:1018E000232B31F08F3F31F481E09F3F19F403C087
:1018F00081E001C080E080FD47C04F815885698547
:101900007A858B859C850E94F7073EC086E0FE01A4
:101910003796DE01119601900D928A95E1F7FF81CD
:10192000E8856A857B856115710531F0EF3F31F4FB
:1019300081E0FF3F19F403C081E001C080E080FD39
:1019400023C02091170230E0C901019687709927C2
:101950004091160250E084179507F1F1F983EA836C
:101960007D836C8396E0929FD001939FB00D1124EC
:10197000A85EBD4FFE01319601900D929A95E1F758
:10198000809317020E94DE0916E080911602909162
:101990001702891771F1189FC0011124885E9D4FAD
:1019A0000E94850A882329F1E09116021E9FF0010A
:1019B0001124E85EFD4F40815181628173818481F1
:1019C00095810E94F7078091160290E0019687703A
:1019D000992780931602D9CF0E94C107109217024F
:1019E00010921602E8E4F2E086E0DF011D928A958B
:1019F000E9F72C960FB6F894DEBF0FBECDBFDF918E
:101A0000CF911F9108958091560285958595859572
:101A100008958091560287700895909156029770AC
:101A200081E009F480E00895809161020895909129
:101A30006102892B809361020895809590916102E3
:101A40008923809361020895109261020895909114
:101A50006002892B809360020895809590916002C6
:101A60008923809360020895109260020895809106
:101A70005702089508950C943A0D0C943B0D9091E3
:101A8000B20292FD08C090915702981721F08093FE
:101A900057020C943D0D089580915702882329F038
:101AA0001092570280E00C943D0D0895CF93DF9380
:101AB000E0910201F0910301809161028083E09145
:101AC0000201F0910301908180916002892B808353
:101AD00080915702882381F0E0910201F091030187
:101AE0009081892B808380910201909103010E9453
:101AF000272081110E944C0DC0910201D091030159
:101B000048E050E06EE472E0CE010E94F528892B97
:101B100069F088E0FE01AEE4B2E001900D928A9592
:101B2000E1F7CE01DF91CF910C94E21FDF91CF91CD
:101B300008950C943A0D9091B20292FD10C098E075
:101B4000899F90011124262B209356020E94790828
:101B5000809156028595859585950C94990D0C94E8
:101B600079081092560280E00C94990D209156024B
:101B70008095822380935602982F977099F430E0D5
:101B8000482F082E000C550B2417350759F090915B
:101B9000B20292FD07C08595859585950E949A08A9
:101BA0000C94B10D08959091B20292FB222720F976
:101BB000281769F080FB92F99093B2028091B102EC
:101BC0009091B2020E94210E82E00C94B60D08950D
:101BD0008091B20282FB882780F991E089270C94DA
:101BE000D30D81E00C94D30D80E00C94D30D6FEFF6
:101BF0007FEF80E090E00C94342980E090E00E9438
:101C0000102921E0893E9E4F09F020E0822F08959F
:101C100082E090E00C94022983E090E00C94022989
:101C2000CF9384E090E00E940229C82F82E290E0E6
:101C30000E9402292C2F30E0A901582BCA01CF9114
:101C40000895CF93C92F682F84E090E00E94162951
:101C50006C2F82E290E0CF910C941629AB01BC016D
:101C60008FE090E00C942829AB01BC0183E190E067
:101C70000C94282960E070E0CB010C94340E60E0F5
:101C800070E0CB010E942E0E0C943A0E69EE7EEFAE
:101C900080E090E00E94342960E082E090E00E94C1
:101CA000162960E083E090E00E941629109212024B
:101CB00010921302109214021092150260E084E058
:101CC00090E00E94162960E082E290E00E941629CE
:101CD00060E085E090E00E94162960E086E090E0F8
:101CE0000E9416296FEF87E090E00E94162940E0DD
:101CF00050E0BA0188E090E00E94282960E08DE081
:101D000090E00E94162940E050E0BA0188E190E09E
:101D10000E94282960E087E190E00E94162940E0B7
:101D200050E0BA018CE190E00E94282960E070E068
:101D300080E290E00E94342940E050E0BA0188E15E
:101D400090E00E9428290C943F0E0C94460E682FB8
:101D50008EE090E00C9416290E941C21609374027E
:101D6000709375028093760290937702609370026D
:101D700070937102809372029093730208950E948F
:101D80001C21609374027093750280937602909385
:101D9000770260936C0270936D0280936E02909351
:101DA0006F02089585B7806885BF85B7806885BF55
:101DB000089581E008950C94D90E08950C94DD0ED9
:101DC0000C94DD0E0C94E00E0C94DD0E0C94E40EDD
:101DD0000C94DD0E0E94D20E83EB91E10E94CC1F89
:101DE0000E94E80E0C94E60E0E94DE0E0C94DD0EAE
:101DF0000E94CD110C9408040E9407210E94B21287
:101E00000E94F80E0E94401B0E946E1E0C94E20E6F
:101E10005F926F927F928F929F92AF92BF92CF927A
:101E2000DF92EF92FF920F931F93CF93DF93CDB783
:101E3000DEB72A970FB6F894DEBF0FBECDBF0E9463
:101E4000C712C82E81110E94AC0E32E6832E32E0FA
:101E5000932E00E010E0502E802F0E94F1115C01C3
:101E6000F401619071904F01682679266114710424
:101E7000B1F40F5F1F4F0530110569F78FEF8983AC
:101E80008A831B820E9410218160782F9D838C831E
:101E900049815A816B818D810E9424043AC08091CE
:101EA000780281FD0E94FA11D12CEE24E394F12CEA
:101EB000C3018E219F21892B29F10E94DB0E8823EB
:101EC000A9F0DE825F82AE20BF2081E0AB2809F45A
:101ED00080E088870E9410218160782F9A87898707
:101EE0004E815F8168858A850E942404000F111F3E
:101EF000F801EE59FD4F80819181E826F926F182A3
:101F0000E08207C0D394EE0CFF1CF0E1DF12D0CFCB
:101F1000B0CF81E0C11001C080E02A960FB6F894DE
:101F2000DEBF0FBECDBFDF91CF911F910F91FF900C
:101F3000EF90DF90CF90BF90AF909F908F907F9069
:101F40006F905F9008950E94080F0E94731B0E947B
:101F5000871E81110E94BF0E0E94CE140C9419049A
:101F6000CF93DF930E94DC10EC01811521E59207ED
:101F700008F045C0811530E5930708F094C0883E0D
:101F8000910528F5803E910508F0F8C0883A910542
:101F900070F4853A910508F07CC08130910509F410
:101FA00075C008F4E8C0049708F0E8C0E4C08F3BAF
:101FB000910508F0E0C0C85AD0E0CC0FDD1FC35A2D
:101FC000DE4F0990D881C02DCE019464D8C0811510
:101FD00040E2940758F4811551E0950708F0CEC00F
:101FE0008D3E910508F4C7C09065C9C0C11580E455
:101FF000D80708F4C0C0DF70CE01906AC0C0811558
:1020000025E59207A8F4811534E5930708F095C0FB
:10201000811543E5940708F07BC0811552E59507CB
:1020200008F061C0D82FCC27CE01816F906AA7C07D
:10203000C11589E5D807A0F4C11528E5D20708F035
:1020400082C0C11536E5D30708F095C08C2F0E94D9
:1020500070118F7190E0D82FCC27CE0190628FC085
:10206000C1154AE5D40708F474C0CE019056811515
:10207000904208F080C08D2F8F710E947011DD2773
:10208000D0628F71AE01582BCA0179C081E090E017
:1020900076C0C55AD0E0C557DE4F8881C82FD0E042
:1020A000CE0190646CC074E0969587957A95E1F7BF
:1020B000282F23703C2F337081E090E002C0880FFE
:1020C000991F3A95E2F79C68AC01522B9A019C2F1C
:1020D0009F709695969550E2959FE0011124C90155
:1020E0008C2B9D2B4CC08370992721E030E002C0DF
:1020F000220F331F8A95E2F79C2F9695969580E2E2
:10210000989FE0011124C22BD32BCE019C6837C0CD
:102110008370992721E030E002C0220F331F8A9597
:10212000E2F79C2F9695969540E2949FE00111244A
:10213000C22BD32BCE019A6822C0D82FCC27CE0138
:10214000846F906A1CC0DC2FCC27CE01806F906A10
:1021500016C08C2F8F700E94701194E0D695C79591
:102160009A95E1F7CF70D0E0DC2FCC27D0699E01A3
:10217000282BC90104C080E090E001C0CE01DF91AE
:10218000CF910895E72FF0E095E0899FE00DF11DD4
:10219000112484E0EE0FFF1F8A95E1F7E60FF11D91
:1021A000EE0FFF1FE852FF4F8591949108950E9412
:1021B000C2100E94B00F08958238910569F1B0F401
:1021C0008133910509F46DC048F48932910509F411
:1021D00063C08A32910509F469C008958533910579
:1021E00009F455C089339105B9F00895833E9105EE
:1021F00069F138F4803E9105B1F0823E910509F114
:102200000895863E9105A9F1873E9105B9F1843E76
:10221000910509F064C023C02091B10220FD4FC098
:1022200021FD4DC008958091B10280FD44C0809190
:10223000B20280FF44C08091B10284FD42C083EEAF
:102240004DC08091B10282FF38C0F5CF8091B102BC
:1022500082FD33C08091B20280FD31C0ECCF80910D
:10226000B20281FF32C08091B10284FD2AC087EEA4
:1022700035C08091B10283FF26C0F5CF8091B102B5
:1022800083FD21C08091B20281FD1FC0ECCF8091FF
:10229000B10285FD1CC01DC08091B10285FD19C031
:1022A00016C08091B10286FD16C017C08091B102A0
:1022B00086FD13C010C089E311C082EE0FC080EE0E
:1022C0000DC080E00BC086EE09C084EE07C089E235
:1022D00005C085E303C08AE201C081E390E0089570
:1022E0009091B10292FF0DC0282F2871283019F467
:1022F000877F846006C0282F2471243011F48B7FDF
:10230000886093FF0DC0282F2871283119F4877E2B
:10231000846106C0282F2471243111F48B7E8861DA
:102320002091B20220FF0DC0382F3871383019F4D7
:10233000877F816006C0382F3171313011F48E7F74
:10234000886021FF0DC0282F2871283119F4877E5D
:10235000816106C0282F2171213111F48E7E8861A0
:1023600094FD877E089580E008950C94F70D0E94F7
:10237000C7128FE39CE90197F1F700C000000E94AB
:10238000C71280E00E94F11180FF04C00E94B511C5
:102390000C945D2108950C94B7110E94FD0D8111DC
:1023A00002C00E94A50E0E94080E809378020E942F
:1023B000100E9093B2028093B1020E94CB110E9442
:1023C0000C0E682F70E080E090E00E941908609188
:1023D0000E0270910F0280911002909111020C94E4
:1023E0005108E82FF0E0EE0FFF1FE354FD4F80810E
:1023F00091810895089580EA8A95F1F7089500C0C3
:1024000008950C94FB1108950C9403120C9404127B
:102410000C9403120C940812F894E82FE295EF70D4
:10242000F0E031A1282F2F7081E090E001C0880FEB
:102430002A95EAF7982F9095932391A392A1892B3F
:1024400082A3789408950F931F93CF93DF93CEE9DF
:10245000D1E089918F3F11F00E940C1281E0C33AC4
:10246000D807B9F7CEE8D1E00EE911E089918F3FA6
:1024700011F00E940C120C171D07C1F7DF91CF91CC
:102480001F910F910895BF92CF92DF92EF92FF922A
:102490000F931F93CF93DF938C01C62FD0E0CE0113
:1024A00082569E4F6C01FC0190819F3F09F450C001
:1024B000B62EF894E92FE295EF70F0E081A19F70BD
:1024C00021E030E001C0220F9A95EAF7822B81A328
:1024D00082A12095282322A378940E94FF11EEE880
:1024E000F1E04EE951E021E030E0E12CF12C619186
:1024F0006F3F89F0A62FA295AF70B0E090968C91B7
:1025000090E06F7002C0959587956A95E2F780FD1F
:1025100002C0C90102C080E090E0E82AF92A220F37
:10252000331F4E175F0719F7F60180818F3F11F0B7
:102530000E940C1261E0E114F10409F460E08B2DBB
:102540000E940112CC0FDD1FC00FD11FF982E8825B
:10255000DF91CF911F910F91FF90EF90DF90CF907F
:10256000BF9008950E9423128AE0EDEBF2E0DF01B4
:10257000982F1D929A95E9F7E3EBF2E0DF011D92A7
:102580008A95E9F785E00E9412130C948C03FF9260
:102590000F931F93CF93DF93CDB7DEB72A970FB674
:1025A000F894DEBF0FBECDBF8E010F5F1F4F8AE0D4
:1025B000F80111928A95E9F7F12C6F2DC8010E945C
:1025C0004312F394F5E0FF12F8CF4AE050E0B8016F
:1025D00083EB92E00E94F528FF24F394009709F41E
:1025E000F12C892B41F08AE0F801A3EBB2E00190D5
:1025F0000D928A95E1F72F2D45E06DEB72E083EBAC
:1026000092E00E9413130E948E038F2D2A960FB61C
:10261000F894DEBF0FBECDBFDF91CF911F910F9118
:10262000FF9008950895FF920F931F93CF93DF9328
:10263000F82E092F162FD72FC42F222349F081E01F
:1026400080937B020E94102190937A0280937902FA
:1026500080917B028823D9F08091790290917A024F
:102660000E942821059798F0EF2DF02FA12FBD2F64
:1026700080E090E04C2F50E08417950734F42191CE
:1026800031912D933D930196F7CF10927B02DF910C
:10269000CF911F910F91FF9008950E9413230E94E4
:1026A000FC0E0C941F230E9423230E94A30F0C9462
:1026B0003D230E94AE200E94FA220E94EA0E0E9450
:1026C0004D130E9453130E94F40EFBCF809182029F
:1026D00080FF06C06091090170E0660F771F26C079
:1026E00081FF04C06091090184E005C082FF07C03A
:1026F0006091090188E0689FB001112417C0909192
:1027000081029923D1F060910801961788F72091F2
:10271000090188E0289F90011124929FA001939FB6
:10272000500D112470E0CA010E946F2860387105B5
:1027300040F46115710519F406C068E070E0862F59
:1027400008958FE7089581E008958091820280FFC7
:1027500008C06091050170E075956795759567955E
:1027600021C081FF06C06091050170E075956795F5
:1027700019C082FF04C06091050170E010C0909103
:102780008002992399F0609104019617A0F7809137
:102790000501899FC001112470E00E946F286038F4
:1027A000710540F46115710519F406C061E070E02F
:1027B000862F08958FE7089581E008958D3E21F4D6
:1027C0000E946613819504C08E3E29F40E94661310
:1027D0008093860208958F3E21F40E9466138195AE
:1027E00004C0803F29F40E946613809385020895F7
:1027F000893F19F40E94A51305C08A3F31F40E9455
:10280000A51381958093870208958B3F21F40E9440
:10281000A513819504C08C3F29F40E94A5138093D1
:10282000880208959FE0980F983078F421E030E016
:10283000A90102C0440F551F9A95E2F7CA01909171
:102840008402892B8093840208958D3F21F4809126
:10285000820281600BC08E3F21F4809182028260EF
:1028600005C08F3F29F480918202846080938202A8
:1028700008958D3E39F49091860297FF35C01092ED
:10288000860259C08E3E29F4909186021916BCF337
:102890002BC0909185028F3E29F497FF25C010929E
:1028A000850249C0803F19F41916CCF31DC09091E0
:1028B0008702893F29F41916BCF4109287023BC0A5
:1028C0008A3F19F497FF10C0F8CF8B3F39F49091ED
:1028D000880297FF09C0109288022DC08C3F21F416
:1028E000909188021916BCF39FE0980F983080F4FD
:1028F00021E030E0A90102C0440F551F9A95E2F78C
:10290000CA0180959091840289238093840213C028
:102910008D3F21F4809182028E7F0BC08E3F21F487
:10292000809182028D7F05C08F3F29F480918202C1
:102930008B7F8093820280918502811106C08091F5
:102940008602811102C0109281028091870281115A
:1029500006C080918802811102C010928002089501
:102960000E94102120918502211104C0209186022D
:10297000222321F090937F0280937E022091870290
:10298000211104C020918802222321F090937D021E
:1029900080937C0283E892E00C94ED1FEF92FF920B
:1029A0000F931F93CF93DF9300D000D000D0CDB70B
:1029B000DEB786E0E3E8F2E0DE01119601900D92C9
:1029C0008A95E1F7E0908502F090860200918702F7
:1029D000109188021092850210928602109287024E
:1029E00010928802E11003C0FF2009F45DC08091BD
:1029F0007E0290917F020E942821AC019091810279
:102A0000992339F020910A0130E02417350758F056
:102A10004BC020910B018AE0289F900111242417BC
:102A2000350718F041C09F3F19F09F5F90938102D6
:102A3000EE2061F00E9466131E1414F09FEF01C097
:102A400091E0989F902D112490938502FF2061F0D2
:102A50000E9466131F1414F09FEF01C091E0989F2D
:102A6000902D112490938602309185023323E1F05A
:102A7000209186022223C1F045EB3403C0011124CA
:102A8000992319F09093850203C081E08093850219
:102A900035EB2303C0011124992319F0909386028A
:102AA00003C081E080938602011103C0112309F461
:102AB0005DC080917C0290917D020E942821AC0132
:102AC00090918002992339F02091060130E024177B
:102AD000350758F04BC0209107018AE0289F9001EC
:102AE00011242417350718F041C09F3F19F09F5F4C
:102AF00090938002002361F00E94A513101614F039
:102B00009FEF01C091E0989F902D11249093870230
:102B1000112361F00E94A513111614F09FEF01C05C
:102B200091E0989F902D1124909388023091870214
:102B30003323E1F0209188022223C1F045EB3403D6
:102B4000C0011124992319F09093870203C081E0FA
:102B50008093870235EB2303C0011124992319F0D8
:102B60009093880203C081E080938802809185025F
:102B700081110BC080918602811107C0809187026C
:102B8000811103C08091880281110E94B014EB82F0
:102B9000FC820D831E8386E0FE013196A3E8B2E03D
:102BA00001900D928A95E1F726960FB6F894DEBF54
:102BB0000FBECDBFDF91CF911F910F91FF90EF908E
:102BC0000895E3E8F2E086E0DF011D928A95E9F7D7
:102BD0001092810210928002109282020895EF9268
:102BE000FF920F931F93CF93DF938B01682F1111E7
:102BF0000AC0442329F0E82FF0E0E153FC4F649130
:102C0000762F862F75C0212F30E0E82FF0E0442387
:102C100021F0E153FC4FE491F0E046E0049FC00155
:102C20001124CFEFD0E0BE010E945B284BEA46039F
:102C3000C001479F900D1124800F911D800F911DA1
:102C4000982F990F890FAE01421B530B4E9FD00155
:102C50004F9FB00D5E9FB00D11249B2F189FA001B8
:102C60001124452F55278E01041B150B0E9FA00123
:102C70000F9F500D1E9F500D11247E01E81AF10880
:102C8000E29E8001E39E100DF29E100D1124212F73
:102C90003327C21BD30BCE9F9001CF9F300DDE9FF9
:102CA000300D112462307105A9F048F461157105E9
:102CB00069F061307105C9F48B2F752F0DC0643038
:102CC000710581F058F06630710579F47E2F8B2FF5
:102CD000932F0DC0832F7B2F9E2F09C08E2F7B2F0C
:102CE000952F05C08E2F732F02C07E2F852F692F41
:102CF000DF91CF911F910F91FF90EF90089541E0E8
:102D00000E94EF15089508950E947F160895CF93AD
:102D1000DF93762FE901682F842F0E948416798330
:102D200068838A83DF91CF9108958091C702282F0D
:102D3000269530E02115310519F48170826005C0B7
:102D40002532310524F0817088648093C70208958C
:102D500088E090E00C940A29CF92DF92EF92FF92E4
:102D60006B017C010E949516B701A60188E090E0F6
:102D7000FF90EF90DF90CF900C942829E7ECF2E0E1
:102D800083E0808311828FEF82838383148260814A
:102D90007181828193810C94AC168091C70280FF6F
:102DA00002C08695089580E008959091CB029330FB
:102DB00018F49F5F9093CB02882351F06091C70273
:102DC0007091C8028091C9029091CA020C94AC160D
:102DD000089581E00C94D5169091CB02992319F0B7
:102DE00091509093CB02882351F06091C70270916B
:102DF000C8028091C9029091CA020C94AC16089541
:102E000081E00C94EC1670E00C94F01C60911001C1
:102E10008091C70280FF0AC080910F0123E0829F4A
:102E2000C001112484539D4F0C940317809111010C
:102E300090911201891780F7E82FF0E09F01220F8F
:102E4000331FE20FF31FE453FD4F118210821282F1
:102E50008F5FF0CF9091C70290FF16C09091110143
:102E600020911201921770F4E92FF0E0DF01AA0F10
:102E7000BB1FEA0FFB1FE453FD4F81836083428336
:102E80009F5FF0CF0C9406170895CF93DF9300D087
:102E90001F92CDB7DEB79091C70290FF0AC09E0186
:102EA0002F5F3F4F0E9487164B8169818A810E9464
:102EB0002A170F900F900F90DF91CF910895CF9325
:102EC000DF93EC01EC81F0E0E653FD4F4491E7EC39
:102ED000F2E0628181810E9445178C818F5F8C8333
:102EE000DF91CF910895CF93DF93EC01E7ECF2E00F
:102EF000438162818C810E9445178C818F5F8C8316
:102F0000DF91CF9108950F931F93CF93DF9300D05C
:102F10001F92CDB7DEB78C018091890281110AC062
:102F20009E012F5F3F4F4FEF6FEF0E9487168A8100
:102F300080938902F8018481813051F028F0823039
:102F400061F4409189020AC08091890240E007C083
:102F50006091890240E080E003C040E080E060E0F2
:102F60000E942A17F801848190E0019663E070E0E6
:102F70000E946F2884830F900F900F90DF91CF9164
:102F80001F910F910895AF92BF92CF92DF92EF926F
:102F9000FF920F931F93CF93DF9300D01F92CDB773
:102FA000DEB7182FF62E042FE22E9091C70290FF65
:102FB0006DC0E92FE695AE2FB0E0AD55BE4F8C91B8
:102FC000809393029E7F923061F49E012F5F3F4F6A
:102FD000812F0E9487164B8169818A810E942A175E
:102FE00043C0823019F40091CA023EC0863019F401
:102FF0001091C80239C08930D9F38931A9F5E95156
:103000008E2F8170D82EE695F0E0E653FC4FA59008
:10301000B490C12CBB2460911301C61618F52C2D59
:1030200030E0A29EC001A39E900DB29E900D11248F
:1030300070E00E945B28812FD11002C0860F01C072
:10304000861B90911101290F311DA901440F551FB5
:10305000240F351F24533D4F402F6F2D0E9487169C
:10306000C394D9CF0E9406171093C802F092C902E8
:103070000093CA02EE2051F06091C7027091C8021D
:103080008091C9029091CA020E94AC160F900F90D5
:103090000F90DF91CF911F910F91FF90EF90DF90F4
:1030A000CF90BF90AF900895E7ECF2E09181282F88
:1030B0004381628188E0890F0C94C31781E00C94EE
:1030C0005418E7ECF2E09181282F4381628188EF68
:1030D000890F0C94C31781E00C946118E7ECF2E0BF
:1030E000628121E1620F08F46FEF282F4381818113
:1030F0000C94C31781E00C946E18E7ECF2E0628147
:1031000021E1621B08F460E0282F438181810C9447
:10311000C31781E00C947D18E7ECF2E0438121E1D4
:10312000420F08F44FEF282F628181810C94C3175E
:1031300081E00C948C18E7ECF2E0438121E1421B22
:1031400008F440E0282F628181810C94C31781E04C
:103150000C949B1820E00C94C317FF920F931F93BD
:10316000CF93DF93EC01F12C0FEF10E0609113018E
:10317000F616F0F4809111012F2D30E0280F311D4B
:10318000C901880F991F280F391F24533D4F70E044
:10319000C8010E946F28962F8C814091CA026091CD
:1031A000C902F99E800D11240E948716F394DECF88
:1031B0000E9406179A818C8190FF02C08F5F01C028
:1031C00081508C83DF91CF911F910F91FF900895D3
:1031D000AF92BF92CF92DF92EF92FF920F931F9325
:1031E000CF93DF93FC01828180FF02C00FEF01C00B
:1031F00001E010E048E1A42E80911301181708F0B7
:1032000043C080911101C12ED12CE601C80FD11D00
:10321000CE01880F991FC80FD91FC453DD4F1982E3
:1032200018821A8234E0E32EF12CB12C80918B02AB
:103230008B0D89312CF06A2D0E944D28892F05C0F5
:1032400087FF03C090911301890F082E000C990B82
:10325000C816D90691F48091CA028E9DA0018F9D57
:10326000500D112455954795559547959E016091B0
:10327000C9028091C8020E948716B00EF1E0EF1AD1
:10328000F108A1F61F5FB8CF0E94061780918B024C
:10329000013031F4811102C080911301815007C0C7
:1032A00090E001966091130170E00E946F28809376
:1032B0008B02DF91CF911F910F91FF90EF90DF90E4
:1032C000CF90BF90AF900895CF93809111019091CE
:1032D0001201891770F4E82FF0E09F01220F331FCD
:1032E000E20FF31FE453FD4F1182108212828F5FB1
:1032F000F0CFC0E060911301C617C0F5EC2FF0E0ED
:1033000070E0CF010E946F2820911101820F20915F
:103310008A02022E000C330B90E0E217F307CCF088
:1033200020910E01022E000C330B2E173F078CF05C
:103330009C01220F331F820F931F9C0124533D4F8A
:103340004091CA026091C9028091C8020E9487160A
:103350000BC0FC01EE0FFF1F8E0F9F1FFC01E453FB
:10336000FD4F118210821282CF5FC4CF0E940617D8
:1033700020910D0180918A02820F80938A029091A0
:103380000E01920F90930E0119165CF4082E000C9A
:10339000990B4091130150E0415051098417950752
:1033A0001CF0219520930D01CF9108958F929F924B
:1033B000AF92BF92CF92DF92EF92FF920F931F9343
:1033C000CF93DF938C01FC014481C42FD0E09E0198
:1033D000DE010E94B3289B01AC010E94C9286B0149
:1033E0007C01E0E2F0E0EC1BFD0BA5E5B0E09B0109
:1033F000AC010E94C9284B015C019F01DF010E94C2
:10340000AB289B01AC010E94D4289B01AC012C0D80
:103410003D1D4E1D5F1DC501B4010E948328C22FB2
:10342000D22F2A3228F4F3E02F9F900111240DC0EF
:1034300025E530E02C1B3109C901880F991F280FA1
:10344000391F37FF02C02F5F3F4F35952795C22F99
:10345000C095F12C85E5E82EED1A80911301F81640
:10346000C8F4F1FC02C08E2D01C08D2F9091110186
:103470002F2D30E0290F311DA901440F551F240FB6
:10348000351F24533D4F4C2F6091C9020E9487166F
:10349000F394E3CF0E940617F8018481811102C0E2
:1034A00091E003C0803219F49FEF90930C0190914A
:1034B0000C01890FF8018483DF91CF911F910F9147
:1034C000FF90EF90DF90CF90BF90AF909F908F9044
:1034D00008950F931F93CF93DF93EC0100E010E06A
:1034E00080911301282F30E00217130724F59091E3
:1034F00011019801290F311DA901440F551F240FF7
:10350000351F24533D4F869590E04C8108171907CD
:103510001CF4442331F002C0411103C04091CA029F
:1035200001C040E06091C9028091C8020E948716E4
:103530000F5F1F4FD5CF0E9406178C8190E0019638
:10354000817099278C83DF91CF911F910F910895FE
:10355000E7ECF2E080818E7F8083608171818281DF
:1035600093810E94AC16109294022FEF80E792E0B4
:10357000215080409040E1F700C000000C940617F5
:103580006091C702669570E04BE050E084E191E005
:103590000E94E828892B19F481E0809394020E940C
:1035A000102190938D0280938C0208959091C70210
:1035B00090FF35C09170811102C0926006C08532C3
:1035C00010F0986402C0880F982B9093C70266236E
:1035D00051F06091C7027091C8028091C902909128
:1035E000CA020E94AC166091C702669570E04BE07B
:1035F00050E084E191E00E94E828892B19F01092B4
:10360000940202C00E94C01A81E080938F02409110
:10361000CA026091C9028091C8020C94AA18089548
:10362000682F9091C702969581E0890F853208F046
:1036300081E00C94D61A81E00C94101B682F9091B5
:10364000C70296958FEF890F09F484E20C94D61A7D
:1036500081E00C941E1B61E00C94D61AE7ECF2E0BA
:1036600080818160808386950C942B1B8091C7029A
:1036700080FD0C94A81A0C942E1B60E00C94D61AB2
:103680008091920281112EC00E94FD0D811104C013
:103690000E94A50E0E94BE160E94A8166093C70243
:1036A0007093C8028093C9029093CA026E7F61F43E
:1036B0000E94BE160E94A8166093C7027093C802AB
:1036C0008093C9029093CA020E94951610929402A8
:1036D0008091C70280FF03C086950E943D1B81E058
:1036E0008093920208950F931F93CF93DF9380915D
:1036F0009402882309F485C080919302E091C70267
:10370000E695E81BE0938E02823049F4F0E0EA533C
:10371000FD4FE491CE2FD0E00FE517E149C0863090
:1037200049F4F0E0ED53FD4FE491CE2FD0E003E7F4
:1037300017E13EC0893051F4E695F0E0E054FD4FCA
:10374000E491CE2FD0E00DEA18E132C08F3051F471
:10375000E695F0E0E354FD4FE491CE2FD0E008EE83
:1037600018E126C0853149F4F0E0E654FD4FE491BC
:10377000CE2FD0E004E619E11BC0883181F08332FE
:1037800039F4E8EBF2E0C591D49103E817E110C0F9
:10379000843251F4C4EFD1E009E61AE109C0C8E26D
:1037A000D0E006ED19E104C0C0EDD7E003E816E172
:1037B00080918F02882361F010928F020E94102165
:1037C00090938D0280938C0210929102109290023D
:1037D0000E941021E0918C02F0918D028E1B9F0BB4
:1037E0008F3F9F4770F4EC0FFD1FF0938D02E09325
:1037F0008C028CE892E0F801DF91CF911F910F913C
:103800000994DF91CF911F910F910895882311F0B2
:10381000FA0101C0FB010994CF93DF93C82FD62F83
:103820000E94CD168C1740F00E94CD168D1720F403
:10383000DF91CF910C941B1B8C2FDF91CF910C94B7
:103840002B1B1F93CF93DF93FB0112811111C3C078
:10385000EC010E94140D8272CD3CFCE5DF0709F4F7
:103860009AC0A8F5C73CECE5DE0709F476C0A8F4D9
:10387000C43C9CE5D90709F45FC028F4C33CDC458F
:1038800009F457C054C0C53C9CE5D90709F459C098
:10389000C63CDC4509F45CC04AC0CA3CFCE5DF0715
:1038A00009F46AC050F4C83CECE5DE0709F45AC0DC
:1038B000C93CDC4509F45BC03AC0CB3C9CE5D90768
:1038C00009F45FC0CC3CDC4509F460C030C0C23DA7
:1038D000FCE5DF0709F46FC088F4CF3C9CE5D9070D
:1038E00009F460C008F45CC0C03DFCE5DF0709F4E2
:1038F0005CC0C13DDC4509F45BC019C0C53D9CE519
:10390000D90709F460C050F4C33DFCE5DF0709F4B2
:1039100055C0C43DDC4509F454C009C0C63D9CE512
:10392000D90709F455C0CE35DD4509F454C011E07E
:1039300052C00E94361B4FC048E25BE16BE17BE165
:1039400004C04BE15BE168E27BE10E94061C43C0DE
:103950004BE658E16EE578E1F8CF4EE558E16BE6CD
:1039600078E1F3CF49E858E16AE778E1EECF4AE73A
:1039700058E169E878E1E9CF47EA58E168E978E198
:10398000E4CF48E958E167EA78E1DFCF40E057E16A
:1039900069EE76E1DACF49EE56E160E077E1D5CF26
:1039A00081E017C065E082E010C068E086E00DC0ED
:1039B0006EE089E00AC064E18FE007C067E185E15D
:1039C00004C088E106C062E289E10E940C1C03C0C9
:1039D00083E20E942B1B812FDF91CF911F910895CD
:1039E0006E9A2EB12F7B3EB130644FB7F894FC0134
:1039F000CB01880F991F680F791F6E0F7F1FE61785
:103A0000F70789F0819198E03EB9000000C087FF78
:103A10002EB9880F000000C000C000C02EB900C041
:103A20009A9591F7ECCF4FBF8FE594E00197F1F7AE
:103A300000C000000895CF93DF93EC01FB01828169
:103A4000882309F43CC1C430FDE5DF0760F4CB3FB7
:103A50009CE5D90788F49E0122503C45243131056C
:103A600008F02EC109C0C236EDE5DE0729F0C63ADE
:103A7000FDE5DF0709F024C10E94100E9093B20209
:103A80008093B102C1318CE5D80709F4C6C008F0B3
:103A900042C0C930ECE5DE0709F49BC000F5C53033
:103AA0008CE5D80709F485C078F4C330ECE5DE076F
:103AB00009F478C008F07AC0C230DC4509F0F5C0DE
:103AC0008091B1028160EFC0C7309CE5D90709F44D
:103AD00078C008F07AC08091B1028061E4C0CD3036
:103AE000FCE5DF0709F487C058F4CB309CE5D90723
:103AF00009F479C008F07BC08091B10288606FC082
:103B0000CF30FCE5DF0709F480C008F082C0809167
:103B1000B102877FC8C0CE3F9CE5D90709F471C0C8
:103B200000F5C531FCE5DF0709F485C068F4C33151
:103B30009CE5D90709F475C008F095C00E94C1073B
:103B40008091B1028F77AFC0CC3FFCE5DF07A9F1D0
:103B500008F054C0CB3FDC4509F0A7C08091B20209
:103B600040C0C230EDE5DE0709F489C058F4C11544
:103B70008DE5D80709F45AC008F069C08091B202F7
:103B800082602FC0C236EDE5DE0709F47CC0C63A7C
:103B9000FDE5DF0709F481C0C330DD4509F085C0CC
:103BA00080E06EC08091B10282607DC08091B102E0
:103BB00016C08091B102886076C08091B2028260A6
:103BC0004FC08091B10280626EC08091B10280646A
:103BD0006AC00E94C1078091B102806864C084609D
:103BE00062C081603DC08091B1028E7F5CC08091D7
:103BF000B1028D7F58C08091B10216C08091B2028F
:103C000018C08091B2028D7F2BC08091B1028F7E4F
:103C10004AC08091B1028F7D46C08091B1028F7BF6
:103C200042C08091B102877F8B7F3DC08091B202FC
:103C30008D7F8E7F15C08091B10282FB222720F9F3
:103C400091E0922790FB82F990FB83F92CC0809140
:103C5000B202982F909591708E7F892B90FB81F9FD
:103C60008093B20222C00E94C1078091B10287FBFB
:103C7000222720F991E0922790FB87F914C081E078
:103C80000E94A70E12C08091B10284FB222720F966
:103C900091E0922790FB84F906C08091B102982FA1
:103CA000909590FB80F98093B1028091B102909140
:103CB000B2020E94210E0E94C10780E001C081E093
:103CC000DF91CF9108958FE891E00197F1F700C05F
:103CD0000000089581E008950C946A1E23982B9AA1
:103CE00027982F9A0E94631E83B183FB882780F94F
:103CF00023B130E0220F232F221F330B232B11F48B
:103D000090E001C092E0892B809397020895E091A2
:103D10009702EE0FEE0FE093970223B123FB882763
:103D200080F990E023B130E0220F232F221F330BC4
:103D30002115310511F022E030E0822B932B8E2BE0
:103D4000809397028F70E82FF0E0E853FE4F908148
:103D500080919602890F8093960284305CF0809166
:103D600095028F5F8093950260E080E00E946C1E58
:103D700021E001C020E0809196028D3F54F48091B3
:103D8000950281508093950261E080E00E946C1E54
:103D900021E080919602082E000C990B64E070E0FF
:103DA0000E946F2880939602822F0895CF93DF930D
:103DB00086319C4541F5EB010E94140D982F8A81B4
:103DC0002091020130910301882379F09A7A81E0F1
:103DD00009F480E080939802911102C069E201C069
:103DE00065E3C9010E9469200AC08091980281118F
:103DF00002C069E201C065E3C9010E946B200E9414
:103E0000560D80E001C081E0DF91CF9108950F93BE
:103E10001F93CF93DF93C42FD22FFC01828188237D
:103E2000C9F040939B020E94102190939A028093C4
:103E3000990280E28C0F883008F057C0C77081E08B
:103E400001C0880FCA95EAF7DF91CF911F910F91BA
:103E50000C941E0580919B02481330C080919902FA
:103E600090919A020E942821883C910538F510E231
:103E70001D0FCD17B9F080E28C0F883040F4C77069
:103E800081E001C0880FCA95EAF70E942505183025
:103E900028F581E09D2F977001C0880F9A95EAF769
:103EA0000E941E05802F0E9415051830F0F4D7706F
:103EB00081E001C0880FDA95EAF70AC080E28C0F32
:103EC000883098F4C77081E001C0880FCA95EAF77E
:103ED000DF91CF911F910F910C942505802FDF91D9
:103EE000CF911F910F910C941505DF91CF911F91E8
:103EF0000F9108950F939C01CB01243F4CE53407AB
:103F000031F188F4293DFCE53F07D9F02A3D4CE525
:103F1000340779F1283D3C45A9F506E221EE41EE52
:103F200068ED7CE52BC0263FFCE53F07E1F0A8F0FB
:103F3000273F3C4539F507E225EE46EE67EF7CE585
:103F40001DC007E225EE45EE69ED7CE517C006E2EF
:103F500021EE40EE64EF7CE511C007E225EE44EE71
:103F600065EF7CE50BC006E221EE42EE66EF7CE5F4
:103F700005C008E221E045EE6AED7CE50E94071FDE
:103F800080E008C0FC018281882319F010929B0216
:103F900001C081E00F9108959093D9018093D801D9
:103FA00008959093A1028093A0020895E091A00249
:103FB000F091A102309721F00190F081E02D099459
:103FC00080E00895E091A002F091A102309721F0E5
:103FD0000280F381E02D09940895E091A002F09110
:103FE000A102309739F022E0DC012C930480F581A6
:103FF000E02D0994089520919E0230919F02281788
:10400000390771F090939F0280939E02E091A00285
:10401000F091A102309721F00680F781E02D0994FC
:10402000089520919C0230919D022817390771F064
:1040300090939D0280939C02E091A002F091A102D6
:10404000309721F00084F185E02D09940895FC015A
:10405000329697E080E0915029F021912223D9F304
:104060008F5FF9CF0895662349F0FC0132960896D8
:104070002191621729F0E817F907D1F780E0089538
:1040800081E008959C01FC0132969FEF80E0419110
:10409000461789F09F3F19F4411101C0982F8F5F97
:1040A0008630A9F79F3F39F0F901E90FF11D97FD1F
:1040B000FA956283089508959C012A5F3F4FFC01A1
:1040C0004281461301C01282019682179307B9F705
:1040D00008950C9442200C945C20029626E0FC018A
:1040E00011922A95E9F7089508950C94742083E0BD
:1040F0008093A2020C947520811102C081E001C05E
:1041000082E08093A2020C9475200C947C2081E0C4
:104110008093A2020C9475200C94872008950C942F
:104120008E200C948F200C948E200C948E200C9456
:104130008E20CF930E9495200E94C7120E94932048
:10414000C0E08C2F0E94F111892B29F4CF5FC5307C
:10415000C1F780E001C081E0CF91089508951F92DA
:104160000F920FB60F9211248F939F93AF93BF932B
:104170008091A302811113C08091140390911503C3
:10418000A0911603B09117034196A11DB11D809314
:10419000140390931503A0931603B0931703BF91D4
:1041A000AF919F918F910F900FBE0F901F90189518
:1041B00080911C03843031F10E94F9031092A30214
:1041C00020E488E190E00FB6F894A8958093600011
:1041D0000FBE2093600083B7817F846083BF83B765
:1041E000816083BF7894889583B78E7F83BF0FB635
:1041F000F894A89580916000886180936000109287
:1042000060000FBE08950E94C1070C94FD0382E078
:1042100084BD93E095BD9AEF97BD80936E0008959D
:104220002FB7F8948091140390911503A091160371
:10423000B09117032FBF08952FB7F894609114031E
:104240007091150380911603909117032FBF089565
:104250009C014FB7F8948091140390911503A0919D
:104260001603B09117034FBF821B930B08957894E8
:104270001F920F920FB60F9211248F939F93AF93BB
:10428000BF938091140390911503A0911603B091F0
:1042900017030196A11DB11D80931403909315037C
:1042A000A0931603B0931703BF91AF919F918F9185
:1042B0000F900FBE0F901F90189581E08093E00043
:1042C00080E28093D8001092C9008FE19EE40197AC
:1042D000F1F700C0000087E090EBDC01809325033C
:1042E00090932603A0932703B09328039CE088E1D2
:1042F0000FB6F894A895809360000FBE909360006D
:10430000FFCF8091AF020895089522E02093E90045
:104310002FEF3091E800215035FD06C035ED3A957C
:10432000F1F700002111F5CF2091E80025FF0BC027
:1043300040E050E066E070E00E94AF238091E8002A
:104340008E778093E8000895CF93DF9321E0209348
:10435000E9002FEF3091E800215035FD06C035ED22
:104360003A95F1F700002111F5CF2091E80025FFE3
:1043700014C0EC0140E050E068E070E00E94AF2320
:104380008091E8008E778093E80088E0FE01A7EA3C
:10439000B2E001900D928A95E1F7DF91CF910895F7
:1043A0008093A4027093A6026093A50280911C03DF
:1043B000843001F582E08093E9008FEF9091E8006E
:1043C000815095FD06C095ED9A95F1F70000811199
:1043D000F5CF8091E80085FF0DC040E050E063E03C
:1043E00070E084EA92E00E94AF238091E8008E772B
:1043F0008093E8000895BC0184E00C94D021BC01B6
:1044000083E00C94D02180911B03811109C00E948C
:1044100040250E949D258091E20084608093E20007
:10442000089510921B0308950C948C20609118033A
:1044300081E0611101C080E00C94772090911C0311
:1044400081E0943009F080E0609118030C947C20A6
:1044500042E061EC81E00E94B92442E261EC82E03A
:104460000E94B92490911C0381E0943009F080E00F
:10447000609118030C94852080911E03833009F409
:1044800061C030F4813071F0823009F49AC008952F
:104490008A3009F486C08B3009F46CC0893009F089
:1044A000A8C020C080911D03813A09F0A2C080916C
:1044B000E800877F8093E800809121039091220398
:1044C000892B21F468E087EA92E003C060E080E095
:1044D00090E070E00E94FA238091E8008B7780934F
:1044E000E800089580911D03813209F082C0809117
:1044F000210390912203029708F07BC08091E8008D
:10450000877F8093E8008091E80082FD05C080915C
:104510001C038111F8CF6DC02091F3008091F2004F
:1045200090E0922B029731F48091F100813011F0EC
:10453000863021F48091F1008093AF028091E800F1
:104540008B7753C080911D03813A09F052C080914E
:10455000210390912203892B09F04BC08091E80040
:10456000877F8093E8008091E80080FFFCCF8091F6
:104570002B0136C080911D038132D9F58091210332
:1045800090912203892BA9F58091E800877F809381
:10459000E8000E94EE2480911F0380932B010C946D
:1045A000C10780911D03813221F58091E800877F4A
:1045B0008093E8000E94EE24809120038093B00253
:1045C000089580911D03813AA1F48091E800877FCE
:1045D0008093E8008091E80080FFFCCF8091B002DA
:1045E0008093F1008091E8008E778093E8000C942E
:1045F000EE24089584B7877F84BF0FB6F894A895FA
:1046000080916000886180936000109260000FBE0E
:1046100090E080E80FB6F894809361009093610079
:104620000FBE0C9487200E9440250E949D25E2EE3B
:10463000F0E080818460808378940C9432288FE14C
:1046400091E00C94D11F80911C038530A9F48091D6
:104650001C03853079F40E94D82080911A038823A6
:10466000B1F30E949920882391F30E9499230E941C
:10467000C107EDCF0C940321089508950C944023B5
:10468000292F332723303105C9F060F4213031055B
:1046900081F02230310509F044C08BE390E027EF30
:1046A00034E043C021323105E1F02232310549F1D5
:1046B00038C082E190E022E335E037C099278130AD
:1046C000910549F028F0029761F5EFECF4E005C0A0
:1046D000E3EFF4E002C0EFEDF4E0849190E09F019D
:1046E00024C06115710541F061307105D1F489E094
:1046F00090E022E235E019C089E090E029E035E061
:1047000014C06115710541F06130710551F48BE7FA
:1047100090E024E435E009C080E490E02FEB35E040
:1047200004C080E090E020E030E0FA013183208393
:10473000089580E189BD82E189BD09B400FEFDCF05
:104740008091D8008F7D8093D8008091E0008260B6
:104750008093E0008091E00081FDFCCF0895CF922E
:10476000DF92EF92FF920F931F93CF93DF93EC01B1
:104770008B017A010E940D25811133C0E114F104EF
:1047800039F0F70180819181081B190BC80FD91FDF
:10479000C12CD12C0115110519F18091E80085FD7E
:1047A00016C08091E8008E778093E800E114F10450
:1047B00049F0F70180819181C80ED91ED182C08253
:1047C00085E00FC00E940D25882321F30AC089913E
:1047D0008093F10001501109FFEFCF1ADF0ADACF01
:1047E00080E0DF91CF911F910F91FF90EF90DF90CC
:1047F000CF90089520912303309124032617370783
:1048000048F06115710539F42091E8002E77209366
:10481000E80001C0B901FC0120E06115710579F1E2
:1048200080911C038823F1F18530F1F18091E8003B
:1048300083FD3CC08091E80082FD2EC08091E8009D
:1048400080FFEBCF2091F3008091F20090E0922B5B
:104850006115710551F08830910538F4219120934C
:10486000F100615071090196F3CF21E0089709F03A
:1048700020E08091E8008E778093E800CECF211170
:10488000CFCF0AC080911C03882361F0853061F08E
:104890008091E80083FD0AC08091E80082FFF2CF9A
:1048A00080E0089582E0089583E0089581E008950E
:1048B00020912303309124032617370748F0611510
:1048C000710539F42091E8002E772093E80001C0AB
:1048D000B901FC0120E06115710591F180911C0383
:1048E000882309F440C0853009F43FC08091E80076
:1048F00083FD3DC08091E80082FD2FC08091E800DB
:1049000080FFE9CF2091F3008091F20090E0922B9C
:104910006115710559F08830910540F42491209378
:10492000F1003196615071090196F2CF21E00897AC
:1049300009F020E08091E8008E778093E800CBCFEB
:104940002111CCCF0AC080911C03882361F08530EF
:1049500061F08091E80083FD0AC08091E80082FF49
:10496000F2CF80E0089582E0089583E0089581E029
:104970000895982F973068F59093E900981739F0CB
:104980007091EC002091ED005091F00003C0242FB5
:10499000762F50E021FD02C09F5FECCF3091EB00FD
:1049A0003E7F3093EB003091ED003D7F3093ED0082
:1049B0003091EB0031603093EB007093EC0020936A
:1049C000ED005093F0002091EE0027FDE5CF80E050
:1049D00008958F708093E90081E0089580911D0310
:1049E00087FF11C08091E80082FD05C080911C0303
:1049F0008111F8CF11C08091E8008B770BC08091B6
:104A00001C03882349F08091E80080FFF8CF809153
:104A1000E8008E778093E80008952091E4003091BB
:104A2000E50095E64091EC00842F817040FF23C0A3
:104A30008091E80080FD1DC080911C03882399F0BF
:104A4000853099F08091EB0085FD11C04091E40024
:104A50005091E5002417350729F3915011F09A0180
:104A6000E1CF84E0089582E0089583E0089581E035
:104A7000089580E008954091E80042FFDDCF089559
:104A80000E94AE250E94B625E0EEF0E080818160B4
:104A90008083E8EDF0E080818F77808319BCA7EDFB
:104AA000B0E08C918E7F8C9380818F7E808310927A
:104AB0001B0308950F931F93CF93DF930E94AE259E
:104AC0000E94B625C8EDD0E088818F7788838881E1
:104AD0008068888388818F7D888319BC10921C032D
:104AE0001092180310921A031092190300EE10E0AE
:104AF000F80180818B7F808388818160888342E098
:104B000060E080E00E94B924E1EEF0E080818E7FD9
:104B10008083E2EEF0E08081816080838081886024
:104B20008083F80180818E7F808388818061888383
:104B3000DF91CF911F910F910895E8EDF0E0808112
:104B40008F7E8083E7EDF0E080818160808384E068
:104B500082BF81E080931B030C945A25E8EDF0E0BE
:104B600080818E7F80831092E20008951092DA0097
:104B70001092E10008951F920F920FB60F92112428
:104B80002F933F934F935F936F937F938F939F9355
:104B9000AF93BF93EF93FF938091E10082FF0BC02F
:104BA0008091E20082FF07C08091E1008B7F8093BB
:104BB000E1000E9431288091DA0080FF1FC08091BF
:104BC000D80080FF1BC08091DA008E7F8093DA00CE
:104BD0008091D90080FF0DC080E189BD82E189BD4F
:104BE00009B400FEFDCF81E080931C030E940322E4
:104BF00005C019BC10921C030E9411228091E10093
:104C000080FF19C08091E20080FF15C08091E20012
:104C10008E7F8093E2008091E20080618093E200C9
:104C20008091D80080628093D80019BC85E0809381
:104C30001C030E9416228091E10084FF30C0809105
:104C4000E20084FF2CC080E189BD82E189BD09B406
:104C500000FEFDCF8091D8008F7D8093D800809199
:104C6000E1008F7E8093E1008091E2008F7E80934F
:104C7000E2008091E20081608093E200809118035D
:104C8000882311F084E007C08091E30087FD02C013
:104C900081E001C083E080931C030E941E2280916A
:104CA000E10083FF29C08091E20083FF25C080914D
:104CB000E100877F8093E10082E080931C031092E3
:104CC00018038091E1008E7F8093E1008091E200E3
:104CD0008E7F8093E2008091E20080618093E20009
:104CE00042E060E080E00E94B9248091F00088609A
:104CF0008093F0000E941422FF91EF91BF91AF9139
:104D00009F918F917F916F915F914F913F912F91E3
:104D10000F900FBE0F901F9018951F920F920FB615
:104D20000F9211242F933F934F935F936F937F9331
:104D30008F939F93AF93BF93CF93DF93EF93FF93A3
:104D4000C091E900CF708091EC00D82FD17080FD28
:104D5000D0E81092E9008091F000877F8093F00006
:104D600078940E94D1261092E9008091F00088602A
:104D70008093F000CD2BCF70C093E900FF91EF91AD
:104D8000DF91CF91BF91AF919F918F917F916F9163
:104D90005F914F913F912F910F900FBE0F901F90F9
:104DA00018951F93CF93DF93CDB7DEB7AA970FB6B1
:104DB000F894DEBF0FBECDBFEDE1F3E08091F100CE
:104DC000819323E0E532F207C9F70E943C228091EB
:104DD000E80083FF2EC180911D0390911E03492F8F
:104DE00050E04A30510508F024C1FA01EE59FF4F56
:104DF0000C94A528803821F0823809F01AC108C027
:104E00008091190390911A03992389F082600FC051
:104E1000809121038F70873008F00BC18093E900E7
:104E20008091EB0085FB882780F91092E900909132
:104E3000E800977F9093E8008093F1001092F100D2
:104E4000D1C0282F2D7F09F0F4C0882319F08230BB
:104E500061F0EFC080911F03813009F0EAC0933008
:104E600009F080E080931A032EC080911F03811106
:104E70002AC0809121038F702FEF280F263008F071
:104E8000D8C08093E9002091EB0020FF1CC0933034
:104E900021F48091EB00806214C09091EB0090614E
:104EA0009093EB0021E030E0A90102C0440F551FB0
:104EB0008A95E2F74093EA001092EA008091EB00B5
:104EC00088608093EB001092E9008091E800877F72
:104ED0008093E8000E94EE24ACC08111AAC010911A
:104EE0001F031F778091E3008078812B8093E3007C
:104EF0008091E800877F8093E8000E94EE248091F3
:104F0000E80080FFFCCF8091E30080688093E3009D
:104F1000111102C082E001C083E080931C0389C0AC
:104F20008058823008F085C080911F039091200343
:104F30008C3D53E0950779F583E08A838AE2898383
:104F40004FB7F894DE01139620E03EE051E2E32FE4
:104F5000F0E050935700E49120FF03C0E295EF701A
:104F60003F5FEF708E2F90E0EA3010F0C79601C0DF
:104F7000C0968D939D932F5F243149F74FBF809149
:104F8000E800877F8093E8006AE270E0CE01019636
:104F90000E94FA2316C06091210370912203AE0192
:104FA0004F5F5F4F0E943E23BC01892B09F441C033
:104FB0009091E800977F9093E80089819A810E9400
:104FC00058248091E8008B778093E80032C08038C5
:104FD00081F58091E800877F8093E8008091180335
:104FE0008093F1008091E8008E7772CF811121C00B
:104FF00080911F039091200399270297D4F4809108
:10500000E800877F8093E80080911F038093180356
:105010000E94EE2480911803811106C08091E30064
:1050200087FD02C081E001C084E080931C030E94E0
:1050300028228091E80083FF0AC08091E800877FE2
:105040008093E8008091EB0080628093EB00AA9649
:105050000FB6F894DEBF0FBECDBFDF91CF911F9189
:1050600008950895CF9380911C038823A1F0C091E7
:10507000E900CF709091EC00892F817090FD80E85D
:10508000C82B1092E9008091E80083FD0E94D12690
:10509000CF70C093E900CF91089587FB082E0626B4
:1050A00087FD819567FD61950E94DC280EF491953E
:1050B00007FC81950895AA1BBB1B51E107C0AA1FDD
:1050C000BB1FA617B70710F0A61BB70B881F991FA9
:1050D0005A95A9F780959095BC01CD01089597FB4D
:1050E000072E16F4009407D077FD09D00E945B28A4
:1050F00007FC05D03EF4909581959F4F08957095DB
:1051000061957F4F0895A1E21A2EAA1BBB1BFD01DA
:105110000DC0AA1FBB1FEE1FFF1FA217B307E40796
:10512000F50720F0A21BB30BE40BF50B661F771FEE
:10513000881F991F1A9469F76095709580959095CE
:105140009B01AC01BD01CF010895EE0FFF1F05903B
:10515000F491E02D09940E94B328332312F48A1BA2
:105160009B0B0C94C428A29FB001B39FC001A39FC6
:10517000700D811D1124911DB29F700D811D112490
:10518000911D08950E94B328B7FF0895821B930BC9
:1051900008950E94B328A59F900DB49F900DA49FE1
:1051A000800D911D11240895B7FF0C94C9280E9409
:1051B000C928821B930B0895991B79E004C0991F9D
:1051C000961708F0961B881F7A95C9F78095089561
:1051D000FC014150504030F001900616D1F7319754
:1051E000CF010895882799270895FB01DC0104C0A9
:1051F0008D910190801921F441505040C8F7881BCF
:10520000990B0895F999FECF92BD81BDF89A99271F
:1052100080B50895A6E1B0E044E050E00C943C294C
:10522000A8E1B0E042E050E00C943C29262FF99927
:10523000FECF92BD81BDF89A019700B4021639F0F5
:105240001FBA20BD0FB6F894FA9AF99A0FBE0895C6
:105250000396272F0E9417290E941629252F0E94A6
:105260001729242F0C9417290196272F0E941729FC
:105270000C941629DC01CB01FC01F999FECF06C084
:10528000F2BDE1BDF89A319600B40D924150504004
:08529000B8F70895F894FFCF70
:10529800C8005802280850011E0A14010101020022
:1052A8001800181801191A1B1C1D1E1F2021228105
:1052B80021A4218521FF21FB21842101E200E900AD
:1052C800EA00B500B600B700CD008301CC008A0122
:1052D80092019401210223022402250226022702B8
:1052E8002A02B300B4006F007000818283E200E9F3
:1052F80000EA00B500B600B700CD008301CC008AF3
:105308000192019401210223022402250226022788
:10531800022A02B300B4006F007000818283F56630
:10532800F6F7673635349796949593929190323183
:10533800F4F1F00001020202020606060909090951
:1053480009090F0F0F0F0F0F15151518191919192E
:10535800191919191919232400FF0100010000FF68
:08536800FF0000010001FF003D
:00000001FF
